S027000062696E2F64656D6F70726F675F6E75636C656F5F73746D33326631303372622E737265636D
S3150800200000500020B9210008FF210008012200081D
S315080020100322000805220008072200080000000025
S31508002020000000000000000000000000092200086F
S315080020300B220008000000000D22000831290008C4
S315080020401322000815220008172200081922000882
S315080020501B2200081D2200081F2200082122000852
S315080020602322000825220008272200082922000822
S315080020702B2200082D2200082F22000831220008F2
S3150800208033220008352200083722000839220008C2
S315080020903B2200083D2200083F2200084122000892
S315080020A04322000845220008472200084922000862
S315080020B04B2200084D2200084F2200085122000832
S315080020C05322000855220008572200085922000802
S315080020D05B2200085D2200085F22000861220008D2
S315080020E0632200086522000867220008EE11AA5537
S315080020F008B540F21C00074BC2F200001B1A062B5B
S3150800210000D808BD40F20003C0F20003002BF8D047
S315080021109847F6E71F00002008B540F21C0040F279
S315080021201C03C2F20000C2F200031B1A9B1003EB49
S31508002130D373591000D108BD40F20002C0F2000264
S31508002140002AF8D09047F6E710B540F21C04C2F210
S315080021500004237873B9FFF7CBFF40F20003C0F2FF
S3150800216000032BB142F65810C0F60000AFF300800A
S315080021700123237010BD00BF08B540F20003C0F26A
S3150800218000034BB142F6581040F22001C0F6000099
S31508002190C2F20001AFF3008040F21C00C2F2000058
S315080021A003682BB140F20003C0F2000303B198475D
S315080021B0BDE80840B0E700BF06498D460649074A0C
S315080021C0074B9A42BEBF51F8040B42F8040BF8E7D6
S315080021D004480047005000205C2900080000002041
S315080021E01C000020E92100081F49204A002301E0BD
S315080021F041F8043B9142FBD300F06CFBFEE7FEE797
S31508002200FEE7FEE7FEE7FEE7FEE7FEE7FEE7FEE798
S31508002210FEE7FEE7FEE7FEE7FEE7FEE7FEE7FEE788
S31508002220FEE7FEE7FEE7FEE7FEE7FEE7FEE7FEE778
S31508002230FEE7FEE7FEE7FEE7FEE7FEE7FEE7FEE768
S31508002240FEE7FEE7FEE7FEE7FEE7FEE7FEE7FEE758
S31508002250FEE7FEE7FEE7FEE7FEE7FEE7FEE7FEE748
S31508002260FEE7FEE7FEE7FEE71C00002090000020E0
S3150800227030B587B04FF40030012100F007FA052089
S31508002280012100F0F1F918238DF817300425ADF86F
S31508002290145003238DF816304FF40064C4F2010479
S315080022A0204605A900F010F98DF817500823ADF857
S315080022B01430204605A900F007F94FF4614301934D
S315080022C00023ADF80830ADF80A30ADF80C30ADF89B
S315080022D010300C23ADF80E304FF48844C4F20004D5
S315080022E020460DEB050100F0E3F92046012100F038
S315080022F047FA07B030BD00BF10B504464FF4884012
S31508002300C4F20000202100F04DFA012808D14FF44C
S315080023108840C4F2000000F041FA2070012010BD88
S31508002320002010BD08B5FFF7A3FF08BD4FF46D42A6
S31508002330CEF20002D16801F4E0610423C0F2FA5338
S315080023400B43D360BFF34F8FFEE700BF08B540F2DB
S315080023507D03C2F200031B7813BB40F23800C2F2B9
S315080023600000FFF7C9FF012859D140F23803C2F22D
S3150800237000031B78002B52D000F0D4FA40F28003F9
S31508002380C2F20003186040F27D03C2F20003012284
S315080023901A7040F27C03C2F2000300221A7008BDCC
S315080023A040F27C03C2F200031B781D481844FFF76D
S315080023B0A3FF012823D140F27C03C2F200031A7856
S315080023C00132D2B21A7040F23803C2F200031B7807
S315080023D09A4224D140F27D03C2F2000300221A7009
S315080023E040F23803C2F200035B78FF2B17D140F2A4
S315080023F03803C2F200039B788BB9FFF797FF00F00A
S3150800240091FA40F28003C2F200031B6864339842D3
S3150800241081BF40F27D03C2F2000300221A7008BD94
S315080024203900002008B5FFF791FF08BD00B583B055
S315080024300420012100F018F92023ADF80430032305
S315080024408DF8063010238DF807304FF40060C4F27B
S31508002450010001A900F038F803B05DF804FB00BFDD
S3150800246010B500F05FFA044640F28403C2F2000396
S315080024701B68C31AB3F5FA7F25D340F28803C2F264
S3150800248000031B786BB940F28803C2F200030122ED
S315080024901A704FF40060C4F20100202100F06AF8B7
S315080024A00CE040F28803C2F2000300221A704FF4CF
S315080024B00060C4F20100202100F05EF840F28403B7
S315080024C0C2F200031C6010BD2DE9F001CB7803F0C1
S315080024D00F02164613F0100F1CBF8E7816430B78A2
S315080024E0FBB10768002301254FF00F0C16E005FA2B
S315080024F003F20C88144094420FD19C000CFA04F89D
S3150800250027EA080706FA04F42743CC78282C08BFDC
S31508002510426102D0482C08BF02610133072BE6D975
S3150800252007600B88FF2B21D94768002301254FF048
S315080025300F0C18E003F1080205FA02F20C881440A1
S3150800254094420FD19C000CFA04F827EA080706FA09
S3150800255004F42743CC78282C08BF4261CC78482C51
S3150800256008BF02610133072BE4D94760BDE8F001D3
S31508002570704700BF016170474161704710B44FF45E
S315080025808053C4F202035B6803F00C03042B08D0E3
S31508002590082B0CD09BBB4FF49053C0F27A03036010
S315080025A032E04FF49053C0F27A0303602CE04FF404
S315080025B08053C4F202035A685B68C2F3834202324C
S315080025C013F4803F07D14FF41063C0F23D0303FBB9
S315080025D002F2026018E04FF48053C4F202035B680B
S315080025E013F4003F19BF4FF41063C0F23D034FF4D4
S315080025F09053C0F27A0303FB02F2026004E04FF440
S315080026009053C0F27A0303604FF48053C4F2020376
S315080026105968C1F3031140F20402C2F20002515C88
S31508002620C9B2046824FA01F141605C68C4F3022463
S31508002630145DE4B221FA04F484605C68C4F3C2242D
S31508002640125DD2B2D140C1605A68C2F3813240F2FB
S315080026500003C2F200039B5CDBB2B1FBF3F101613C
S315080026605DF8044B704700BF39B14FF48053C4F28C
S3150800267002039A691043986170474FF48053C4F275
S3150800268002039A6922EA00009861704739B14FF44B
S315080026908053C4F20203DA691043D86170474FF4D5
S315080026A08053C4F20203DA6922EA0000D86170474F
S315080026B030B587B004460D46038A23F440531B04FD
S315080026C01B0CCA8813430382838923F4B05323F06F
S315080026D00C031B041B0C88880A89498902430A4390
S315080026E01343A381A38A23F440731B041B0CAA89F2
S315080026F01343A38201A8FFF741FF4FF46053C4F2C6
S3150800270001039C420CBF049A039AA3891BB2002BAF
S3150800271002EB820202EB8202BDBF2B685B00B2FBB2
S31508002720F3F22968A4BF8900B2FBF1F248F21F53FD
S31508002730C5F2EB13A3FB02135B091D01642003FB1F
S315080027401023A08900B200280BDADB00323348F2E6
S315080027501F51C5F2EB11A1FB0321C1F34211294315
S315080027600AE01B01323348F21F51C5F2EB11A1FBF7
S315080027700321C1F34311294389B2218107B030BD32
S3150800278029B183899BB243F40053838170478389B7
S3150800279023F400531B041B0C838170478088C0F305
S315080027A00800704700880840003018BF01207047AD
S315080027B000B583B00023019300934FF48053C4F20D
S315080027C002031A6842F001021A6059680022CFF61D
S315080027D0FF020A405A601A6822F0847222F4803294
S315080027E01A601A6822F480221A605A6822F4FE02D5
S315080027F05A604FF41F029A601A6842F480321A60CF
S315080028004FF48053C4F2020340F2DC511A6802F412
S3150800281000320092019A01320192009A12B9019A85
S315080028208A42F3D14FF48053C4F202031B6813F4AF
S31508002830003F00D1FEE74FF40053C4F202031A68C2
S3150800284042F010021A601A6822F003021A601A6827
S3150800285042F002021A604FF48053C4F202035A6827
S315080028605A605A6842F400525A605A6842F48062C2
S315080028705A605A6822F47C125A605A6842F4E8127E
S315080028805A601A6842F080721A604FF48053C4F294
S3150800289002031A6812F0007FFBD04FF48053C4F28B
S315080028A002035A6822F003025A605A6842F002028A
S315080028B05A604FF48053C4F202035A6802F00C02BD
S315080028C0082AFAD1FFF7B2FD00F014F803B05DF854
S315080028D004FB00BF08B5FFF76BFFFFF723FDFFF703
S315080028E0BFFDFFF79FFDFAE740F28C03C2F2000333
S315080028F01860704708B54EF21003CEF2000341F691
S315080029003F12C0F201025A604FF46D42CEF2000245
S31508002910F02182F823100020986007221A60FFF73A
S31508002920E3FF08BD40F28C03C2F200031868704743
S3150800293040F28C03C2F200031A6801321A6070472B
S31508002940F8B500BFF8BC08BC9E467047F8B500BF8E
S31108002950F8BC08BC9E467047000000005A
S3150800295C0204060800000000010203040102030435
S3110800296C0607080979210008492100081F
S70508002000D2
